:020000040000FA
:020000001628C0
:08000800FE00030EFF0083124D
:1000100003130408FD000B18B12C0B19C32C7D0829
:1000200084007F0E8300FE0E7E0E090083120313F0
:1000300085018601831603132B308500403086002E
:1000400044309F0000309F00831603136400C330C8
:1000500081008316031328308B008C018D018312DD
:1000600003138C018D01A9018B174A2A0F398207CE
:100070003034313432343334343435343634373444
:1000800038343934413442344334443445344634CA
:1000900008000F398207BB342834E334EA3478345B
:1000A000DA34DB342A34FB34FA347B34D9349334F5
:1000B000E934D334533408000F3982076534673488
:1000C0006D346F34753477347D347F34E534E73400
:1000D000ED34EF34F534F734FD34FF3408000339E0
:1000E0008207BF34DF34FB34FE340800073982074F
:1000F0008034403420341034083404340234013461
:10010000080007398207FF34FF34FF34FF34FF341F
:10011000FF340034083408000739820705340A34F4
:100120000F34143419341E34323464340800820716
:10013000FF34FE34FC34F834F434F234F034EE346A
:10014000EC34E934E834E734E634E434E334E134DD
:10015000E034DE34DC34DA34D834D634D334CF343B
:10016000CC34C334BC34B134A7349C348F3487349A
:1001700078346E346034563449343F3423340C348C
:10018000003408003F08033982071B2B152B0F2B67
:1001900008003F0803398207762972297A29080066
:1001A00055082F040F3982072F2B372B432B542B45
:1001B000622B6F2B772B802B282BC62BF92BB72B81
:1001C000BC2BCB2BCE2BDC2B08003725AF002F0808
:1001D0000319080066160730F9002F038120AF00CD
:1001E000AF1FD028AC01AD010800AB08031908000F
:1001F0005508031D08006830670784002B0880003D
:1002000086242B080D3A03190C29E70A67080A3AD5
:1002100003195529AB010800F9219725D91828247D
:1002200068082E3A0319682168082C3A0319D72167
:1002300068082B3A03195A2468082D3A03196724D1
:100240006808553A0319CB216808473A0319CF21AA
:100250006808533A03196E2168084D3A0319C22001
:1002600068084C3A0319C9206808463A03198021E6
:100270006808483A0319BE216808423A0319C121A7
:100280006808503A03197C2168084E3A03197E2108
:100290006808443A0319B821E701AB010D30862400
:1002A0000A3086243E3086240800AB01E7010D3079
:1002B00086240A30862445308624723086247230A3
:1002C00086240D3086240A3086243E308624080099
:1002D000FC263E2214273E22142708003F08073937
:1002E000CD000800D911D31250260800D911D31619
:1002F00050260800D91508005914FB2B5910FB2B68
:100300009121BD1B01347308C4007408C500750831
:10031000C600FB25E125FA263E2214273E2214279B
:100320000800402543080F39053AF030031DC30586
:1003300097253D08F3003E08F4003F08F500470804
:10034000BA004808BB004908BC007F25BD1B01342A
:100350004A08BD004B08BE004C08BF007308BA0035
:100360007408BB007508BC007F25BD1B0134003438
:100370003F1CBC296616080005230800E330D600A0
:10038000C329E030D6009121BD1B013473308400B5
:1003900003305D2708003F08E200872608003F1869
:1003A000D4295912C22608005916C22608003E2236
:1003B00014273E2214273E2214273E2214273E22D1
:1003C00014270800F201670803190034E7036708DF
:1003D000031900346830670784000008F2003030E9
:1003E000F202031CE2290A3072020318E2297208A1
:1003F0000800C101C201C301E221C304C30EE2210E
:10040000C304C30EE221C204C20EE221C204C20E22
:10041000E221C104C10EE221C104C10E0800013075
:10042000D825D0002830D200520897205002031C53
:100430001E2A03191E2AD20B142A0034520808005F
:10044000661808000F22D20064020319080052083F
:10045000E400D800AE270730F9006616E618352C00
:1004600008000C30CA00F830CB005030CC0000300F
:10047000C7009C30C8004030C90008001930D8259A
:10048000D10099249924992499241930D825D10090
:10049000C5250800AC01AD01AE01D801D901D501D7
:1004A000D401E7010A30FA00FB01FC01E030D6007C
:1004B0004730840006306527FF30C706031D842AB5
:1004C0004030B000B100B200B300B400B500B600D7
:1004D000B700A324A324A324A324A324A324312268
:1004E000E030D6004730840006305D271930C00068
:1004F0000130C100A030C2006830C300F030D60027
:100500004030840004305D2731220030DE0091301D
:10051000DF00B430E0000130CD00AC01AD01AE0130
:100520005912D915661666146615E610FF30E200FA
:1005300087263C30D8003524D8017330B000212301
:10054000D317F7010F22E400E61DAF2A5808F80080
:100550003C30D800DC237808D800D401E611661AB4
:10056000B62A851AB62A0730F9006616D9182B2440
:100570003E22D227661DF42A661CF22A0F22D200E0
:1005800064020319E22AE5000318D52AE509E50A01
:100590005208E400D50803190F30F7000730F900BE
:1005A00066165A24E50BCA2AF22A5208E400D50836
:1005B00003190F30F7000730F90066166724E50BC2
:1005C000D72AF22AE408031DEA2A0730F900661642
:1005D0006724F22A6408283A031DF22A0730F9003A
:1005E00066165A24000020228A23F520E520A42A3A
:1005F000F70803190800F70B0800E6150800F908CA
:1006000003190800F90B0800080066121030A80052
:10061000051286108614A80B082B861008005315A7
:10062000D31053105316D311202B5311D31453103E
:100630005312D315202B5311D31053145316D31523
:100640005026C830D318C1305319C930B100080042
:100650005318152BD3180F2B53191B2B08000130DF
:10066000D500F230B000B1015914D915080002309C
:10067000D5003B30B000B10159146614E6107F2755
:1006800040258D270800D91808000330D5006611D1
:10069000DA30B000D130B100D330B2007330B300E3
:1006A000B401B501BE2708000430D50066119B30A7
:1006B000B0007B30B1002830B2004930B300B40143
:1006C000A82308000530D5007930B0008030D40070
:1006D000B10166157F2740258D27D9100800063007
:1006E000D5009130B0008030D400B101080007304F
:1006F000D500C030D40066106408D800AE270800CA
:100700000030D5007330B0002123D4015910D91026
:1007100066140800D91D08005A08031DDA03FF30CB
:10072000D0000930D82550025102031CA02BC8303C
:10073000DA00D31E9D2BD3125026D918282C08007E
:100740005A08031D0800D31A0800D31650260800C3
:10075000591AB12BBB30B5005330B6005330B70037
:100760000800BB30B5004930B600B7010800CD0A1B
:10077000CD19CD01BE270800591EC22B5912A8233E
:10078000C22608005916A823C22608006610E614DF
:10079000FF30E400202AE330D600D02BE030D60032
:1007A000D4014430840003305D27A324A324A32470
:1007B000A3248030D40008005808D600FC30D60DA1
:1007C000D60DD605D401C0015308C0001F30C005A6
:1007D0004408C1004508C2004608C30040308400F8
:1007E00004305D27A324A324A324A324C030D40071
:1007F0000800D918282CE030D60047308400063095
:1008000065274A08BD004B08BE004C08BF004708DA
:10081000BA004808BB004908BC007F25BD1F1C2C3E
:10082000E030D6004A30840003306527E330D6003C
:100830004730840003306527591C242C4708C40026
:100840004808C5004908C600DA01D9145910080043
:100850003122D91008001B26FB25E125531BE52674
:10086000FA26DD21F826F92608005808D600FC30C3
:10087000D60DD60DD6054030840004306527C01B48
:10088000522CE03053054004D3004108C400420814
:10089000C5004308C600AE27FB25E125FA26DD2169
:1008A000DA0108004030B200B300B400B500B60071
:1008B000B7000800D3171B26FB25E125531BE526AF
:1008C000FA263E2214273E221427DA010800D31309
:1008D0001B26FB25E125531BE526FA263E2214277D
:1008E0003E221427DA010800A500250E36208624B2
:1008F0002E3086242508362086240800A500250EE3
:100900003620862425083620862408008B13A10073
:100910000830A00086179924A10C03188613031C25
:100920008617A00B8B2C992486138B179924992456
:1009300000341E30A200A20B9B2C00340A30A2000F
:10094000A20BA02C0034FE30A300FE30A400000057
:100950000000000000000000A30BA72CA40BA72C94
:1009600000340830CE009E249924061B0310061F75
:100970000314CF0CCE0BB42C9924061F00004F0893
:10098000AB000B100D28E61ED32CE6126208A60061
:100990000830A800A60D03188614031C8610061044
:1009A0000614A80BCA2CAA0AAA1EE42C29080319AB
:1009B000DD2CF60BDD2CF822FF22290876205405C9
:1009C0000319E42C0301E82C3030290784000008C7
:1009D000661E352DA8005C20A600A80CA80CA80C4B
:1009E000A80C28085C20A70029086F202919A70552
:1009F000291DA6050830A800A60D03180516031C1E
:100A0000051286108614A80BFC2C0830A800A70D30
:100A100003180516031C051286108614A80B072D53
:100A2000051286102908A800A80AA90AA919A9016F
:100A3000851A2E2D2C08031D222D2808AC00AD0090
:100A4000AE01352D28082C06031D352DAE0A2E1EAD
:100A5000352D0F30AE002808AD00352D2C080319B8
:100A6000352D28082C060319AC010B110F282D0871
:100A7000031908008B132D08031DAD018B17080007
:100A800003101830B900C001C101C201C301BF0D7C
:100A9000BE0DBD0DC30DC20DC10DC00DB90B512D45
:100AA0000034433084005E25423084005E254130AE
:100AB00084005E25403084005E25472D033000070A
:100AC000B800B819800030300007B800B81B8000AB
:100AD00000341830B900B801BF0DBE0DBD0DB80D02
:100AE0000318762D3C083802031C792D3C08B80207
:100AF0000314C20DC10DC00DB90B6C2D00348E2531
:100B00003C08BF07031C872DBE0A0319BD0A3B081A
:100B1000BE070318BD0A3A08BD070034BC09BB096B
:100B2000BA09BC0F0034BB0F0034BA0A0034BD014F
:100B3000BE01BF01410EAB254108AB25420EAB25DE
:100B40004208AB25430EAB2543080F39BC00BA0160
:100B5000BB01802500340F39BC00BA01BB018025E0
:100B600003103F0DBC003E0DBB003D0DBA0003104D
:100B7000BF0DBE0DBD0D0310BF0DBE0DBD0D03108D
:100B8000BF0DBE0DBD0D802508005108D0003730C7
:100B900084000830D200D00D0318D32D0011840337
:100BA000D20BCB2D003400158403D20BD32D00348F
:100BB000831203139F0099241F151F19DD2D1E0892
:100BC00008007F274025C101C201972532303F022E
:100BD000031C3F08BC00BA01BB010030BD006730F8
:100BE000BE00E830BF007F253D08DB003E08DC008A
:100BF0003F08DD0008000230BD005D30BE007830E7
:100C0000BF0078277F25BD1B092ED9165913D9138C
:100C100008000630BD00B630BE00C030BF007827E7
:100C20007F25BD1B172ED9125917D9130800D912C9
:100C30005913D91708005317D31F292E4A08BD008E
:100C40004B08BE004C08BF0078277F25BD1B013430
:100C5000332E7F274708BA004808BB004908BC006C
:100C60007F25BD1B01347F27BA01BB014D088C20B5
:100C7000BC00D31B3D2E7F253E2E80253D08C400A1
:100C80003E08C5003F08C6005313003400000000B2
:100C90000000061600000000000000000612080018
:100CA00086270530BC006925831203138B130515B5
:100CB0000830D200C20C03188616031C8612462682
:100CC000D20B5A2E4113C1130830D200C10C0318A5
:100CD0008616031C86124626D20B662EC001D31A36
:100CE000C017531A4017D319C0164014C01140152D
:100CF000C0140830D200C00D03188616031C8612DB
:100D00004626D20B7B2E051186128B170034E61671
:100D10000800061586150800061586150000000057
:100D2000000000000000000086110000000000002C
:100D300000000000000006110800861106150000E2
:100D40000000000000000000000086150800000000
:100D50000000000000000000000006150000000078
:100D6000000000000000000006110800E10008304B
:100D7000D200E10D03188615031C8611A726D20B9D
:100D8000B92E08007F275E08BA005F08BB00600824
:100D9000BC0080253230BC0069258C26C030B626C8
:100DA000A7264108B626A7264208B626A7268830D9
:100DB000591A8930B626A7260130591B0230D91B93
:100DC0000C30B626A7269D260800D31FE92ED31384
:100DD0000800D31708001930D825BF00BE01BD0197
:100DE00040252030862442087E2443087E240800C3
:100DF000080008005026C2267F2740258D270D3089
:100E000086240A30862446308624203086241930F1
:100E1000D825D10041087E244208742443087E244A
:100E20001930D825D100C5255108BF00BE01BD012C
:100E300040252030862442087E2443087E24080072
:100E4000831203135608831203178D0083160317AA
:100E50008C130C14831203170C0883120313D7008E
:100E6000831603178C130C14831203170C088312B8
:100E70000313D706031D202F0800831603178C18B1
:100E80003F2F831203178C0083120313560883121B
:100E900003178D00831603178C130C158B13553015
:100EA0008D00AA308D008C148B170C11831603173C
:100EB0008C18582F831203130800D20000083D2716
:100EC000840AD60AD20B5E2F0800D20020278000A9
:100ED000840AD60AD20B662F08005808D600FC30C8
:100EE000D60DD60DD6054030840004305D270800AD
:100EF0004408BA004508BB004608BC000800440886
:100F0000BD004508BE004608BF0008005B08BD00E4
:100F10005C08BE005D08BF0008000430B205B305E0
:100F2000B405B505B605B705410E4920B204410820
:100F30004920B304420E4920B40442084920B504B4
:100F4000430E4920B60443084920B704BB30321988
:100F5000BF30320604300319B2050800BD01BE01DE
:100F60005808BF00BF0A40250430B005B105430E44
:100F70004920B00443084920B1040800BD01BE0166
:100F80004D088C20BF0040250430B505B605B705D7
:100F900042084920B504430E4920B60443084920BD
:100FA000B7040800BA01BB015108BC00BD017B08B1
:100FB000BE007C08BF0080253E08FB003F08FC0007
:100FC000FA0B08000A30BC006925F530420203180C
:100FD000F42FE6304202031CEE2FF92F620A0319A8
:100FE000F92FE20A8726F92F62080319F92FE20385
:0C0FF0008726FB01FC010A30FA00080013
:02400E00023F6F
:00000001FF
